:020000040800F2
:10000000083400209D0100083F0F0008FD0E000885
:100010003B0F0008F90C0008233600080000000020
:1000200000000000000000000000000005010008C2
:10003000FD0C00080000000049010008B92B000871
:10004000B7010008B7010008B7010008491C000803
:10005000B7010008B7010008B7010008B7010008A0
:10006000B7010008B7010008B7010008B701000890
:10007000B7010008B7010008B7010008B701000880
:10008000B7010008B7010008B7010008B701000870
:10009000B7010008B7010008B7010008B701000860
:1000A000B7010008B7010008B7010008B701000850
:1000B000B7010008852C00080D2D0008B7010008C5
:1000C000B7010008B7010008B7010008B701000830
:1000D000B7010008D932000819330008B701000839
:1000E000B7010008B7010008B7010008DFF810D019
:1000F00000F09CFC0048004729420008AFF3008054
:1001000008340020224B19680868B0E8F00F80F32B
:100110000988BFF36F8F4FF0000080F311884EF015
:100120000D0E70470000000006480068006880F36C
:10013000088862B661B6BFF34F8FBFF36F8F00DFE1
:1001400000BF00BF08ED00E0EFF30980BFF36F8F41
:100150000F4B1A6820E9F00F106008B54FF05000FF
:1001600080F31188BFF34F8FBFF36F8F05F0A6FBAD
:100170004FF0000080F31188BDE808401968086856
:10018000B0E8F00F80F30988BFF36F8F704700BFAE
:10019000F0000020EFF3058070470000064880471C
:1001A00006480047FEE7FEE7FEE7FEE7FEE7FEE75C
:1001B000FEE7FEE7FEE7FEE7252C0008ED0000085D
:1001C00040EA01039B0703D009E008C9121F08C0D9
:1001D000042AFAD203E011F8013B00F8013B521E59
:1001E000F9D27047F0B480EA0102D40F4200B2EBBA
:1001F000410F02D20246084611464A0042D0C30DC2
:10020000DDB2C1F3C752AD1A202D35DAC1F31601A4
:1002100041F4000204B15242C5F1200602FA06F18F
:100220002A411044B3EBD05F23D0C4B1012DA0EB21
:10023000C35009DCF0BC4FF0004202EAC352DBB20B
:1002400000F5000000F04FBB400000F1807000EBB3
:10025000C350A0F1807040EAD170490009E049081C
:1002600041EAC071A0EBC35000F50000400800EB6C
:10027000C350F0BC00F02EBB6142012202EB4101F1
:10028000001BF6E7F0BC704781F00041AAE780F060
:100290000040A7E780EA010210B502F000434000E9
:1002A00022D04A001FD0010E01EB1261C0F35600AC
:1002B000C2F3560240F4000042F40002A0FB022008
:1002C00000047F39140400D0401C50EA124001D4CD
:1002D0004000491EC2B20C0604EBD010401C40087E
:1002E000802A02D003E0002010BD20F00100002988
:1002F00000DA0020184310BD30B480EA010202F099
:10030000004530F0004221F0004013D090B1C30D01
:10031000D40DC2F31601C0F31600E41A41F4000133
:1003200040F400027D34914201D3641C00E0490096
:10033000002C02DA30BC002070474FF4000000238C
:10034000914201D3891A034340084FEA4101F7D192
:1003500051B1914202D14FF0004105E002D24FF07D
:10036000010101E06FF0010103EBC450284430BCEF
:1003700000F0B0BA2DE9FE4F804681EA0300C00FBD
:100380000C46009021F0004123F00045B8EB02003C
:10039000A94105D24046214690461C460B460246DE
:1003A00023F00040104347D0270DC7F30A00C3F3E2
:1003B0000A510290401A019040286BDAC3F31300EF
:1003C00040F4801B0098924620B10023D2EB030A30
:1003D00063EB0B0B01985946C0F14002504600F008
:1003E00048FA06460D4650465946019A00F060FA12
:1003F00010EB08006141002487EA115284EAE77398
:100400001A4340D0009A62B3019A012A4FEA075278
:1004100015DC001B61EB02014FF0004202EA0752BB
:10042000CDE90042001C41F5801132462B4600F018
:1004300097FA03B0BDE8F08F40462146F9E7001B6C
:1004400061EB0201001C41F5801300185B4120188C
:10045000A2F5001747EB030140EAD570B6196D41CC
:1004600011E06D084FEA360645EAC0754FEA0752BB
:10047000001B61EB0201001C41F5801149084FEAA5
:1004800030000019514132462B4603B0BDE8F04F11
:1004900000F057BA0098012240000023D0EB02027E
:1004A00063EBE073009821464FEAE074B8EB00007C
:1004B00061EB0401E9E783F000435BE781F0004171
:1004C00058E72DE9FE4F81EA030404F0004421F0CF
:1004D000004100944FF0000B23F0004350EA010468
:1004E0005ED052EA03045BD0C3F30A54C1F30A5549
:1004F0002C44A4F2F3340194A0FB0254C1F3130181
:1005000041F48011C3F3130343F4801301FB02444D
:1005100000FB034E840A970A44EA815447EA835752
:10052000A4FB076802958D0A05FB07854FEA932C0B
:1005300004FB0C542705029D4FEA065847EA16377C
:10054000B5EB08056EEB070C870E920E47EA811794
:1005500042EA8312A7FB0201B6EB0B0164EB000435
:100560002B0D43EA0C335E1844EB1C50DA4651461F
:10057000E7FB0201C5F313044FEA0B3343EA1453BC
:100580004FEA0432019C43EA0603A4F10C040294EE
:10059000009CCDE900B400F0E3F903B0BDE8F08FB2
:1005A00000200146F9E72DE9F04D81EA030404F04B
:1005B000004B21F0004514464FF0000A23F00041A3
:1005C00050EA050220D054EA01021DD0C5F30A57B3
:1005D0000246C5F31303C1F31300C1F30A5640F4F6
:1005E000801543F48013A7EB0608101BD64608F2CB
:1005F000FD3873EB050002D308F1010801E0921801
:100600005B41B8F1000F03DA00200146BDE8F08D30
:1006100000204FF48011064684460EE0171B73EB52
:10062000050705D3121B63EB050306434CEA010CD7
:1006300049084FEA300092185B4150EA0107EDD1BA
:1006400052EA030012D082EA040083EA050108435B
:1006500005D0101BAB4106D20122002306E0002288
:100660004FF0004302E06FF0010253101AEB060056
:100670004CEB085110EB0A0041EB0B01BDE8F04DCB
:1006800000F05FB9C10F80EAE0700844CA07962302
:10069000002100F028B90EB5C10F80EAE0700844CF
:1006A000CA07002140F233438DE80E000A460B468C
:1006B00000F056F903B000BD0EB540F2334102918F
:1006C0000021CDE900110A460B4600F049F903B0BC
:1006D00000BD20F00040C10DC0F3160040F4000042
:1006E0007F2901DA00207047962903DCC1F19601C9
:1006F000C8407047963988407047C1F30A5210B518
:10070000C1F3130140F2FF3341F480119A4201DA40
:10071000002010BD40F233439A42A2F2334203DC80
:10072000524200F0B5F810BD904010BD00F00042FC
:1007300030F000400AD0C10D01F56071C0F3160021
:1007400042EA0151C20840071143704700200146A8
:100750007047000030B5041E71F1000404DB4FF057
:100760000044404264EB0101141E73F1000405DBF8
:100770001C464FF00043524263EB0403994208BF0A
:10078000904230BD01F0004330B421F0004150EA06
:10079000010206D00A0DA2F56072C1F31301002A0E
:1007A00002DC30BC00207047440F44EAC104C100A1
:1007B000E01830BC00EBC25000F08CB8002801DB20
:1007C000C0F10040002901DBC1F1004181427047C6
:1007D000002801DBC0F10040002901DBC1F100412C
:1007E0008842704730B50B46014600202022012484
:1007F00009E021FA02F59D4205D303FA02F5491BEF
:1008000004FA02F52844151EA2F10102F1DC30BD04
:100810002DE9F05F0546002092469B468846064635
:10082000814640241BE0284641464746224600F0C8
:100830002FF853465A46C01A914110D31146184614
:10084000224600F016F82D1A67EB01084F462246A3
:100850000120002100F00DF817EB00094E41201E89
:10086000A4F10104DFDC484631462A464346BDE890
:10087000F09F202A04DB203A00FA02F100207047A2
:100880009140C2F1200320FA03F3194390407047CE
:10089000202A04DB203A21FA02F00021704721FAD5
:1008A00002F3D040C2F1200291400843194670473C
:1008B000202A06DBCB17203A41FA02F043EAE07324
:1008C00006E041FA02F3D040C2F120029140084311
:1008D000194670470029A8BF7047401C490008BF4F
:1008E00020F00100704710B4B0FA80FC00FA0CF060
:1008F00050EA010404BF10BC704749B1CCF1200498
:1009000021FA04F411FA0CF118BF01212143084324
:10091000A3EB0C01CB1D4FEA00614FEA102042BF50
:10092000002010BC704700EBC35010440029A4BF46
:1009300010BC7047401C490008BF20F0010010BCEB
:10094000704710B5141E73F1000408DA401C41F121
:10095000000192185B411A4301D120F0010010BD43
:100960002DE9F04D92469B4611B1B1FA81F202E0B9
:10097000B0FA80F220329046FFF77BFF04460F4624
:1009800040EA0A0041EA0B0153465A46084313D095
:10099000114653EA010019D0C8F140025046FFF752
:1009A00077FF05460E46504659464246FFF761FF1F
:1009B000084305D0012004E020463946BDE8F08D0B
:1009C0000020054346EAE0762C4337430A98630546
:1009D000E40AA0EB08000022FD0A44EA47540A306A
:1009E00002D500200146E9E7010510196941DDE95A
:1009F000084500196941BDE8F04DA2E7C1F30A526C
:100A0000C1F3130140F2FF3341F480119A4202DA3C
:100A100000200146704740F233439A42A2F233422B
:100A200002DC5242FFF734BFFFF723BF064C074DED
:100A300006E0E06840F0010394E8070098471034AE
:100A4000AC42F6D3FFF756FBB4670008D467000842
:100A500070B58C1810F8015B15F0070301D110F880
:100A6000013B2A1106D110F8012B03E010F8016BAD
:100A700001F8016B5B1EF9D12B0705D40023521E30
:100A80000DD401F8013BFAE710F8013BCB1A921C98
:100A900003E013F8015B01F8015B521EF9D5A14296
:100AA000D8D3002070BD000070B5D37803701379DF
:100AB0000B800B88022B08D1547903785B1E03EB63
:100AC000C3035B00DB1C154DEC540B88032B08D1D2
:100AD000547903785B1E03EBC3035B001B1D0F4DB2
:100AE000EC540B88042B17DB0B88082B14DC55798E
:100AF0000B885B00DB1E0478641E122606FB0433A1
:100B0000064CE55495790B885B009B1E0478641EA7
:100B100006FB0433014CE55470BD00001A000020B0
:100B20002DE9F04307ACF0CC90F800C0ACF1010C1B
:100B30000CEBCC0C4FEA4C0C0CF1030CDFF84C81A5
:100B400018F80CC081F800C090F800C0ACF1010C9E
:100B50000CEBCC0C4FEA4C0C0CF1040C18F80CC04C
:100B600082F800C090F800C0ACF1010C0CEBCC0C8A
:100B70004FEA4C0C0CF1060C18F80C8090F800C0F1
:100B8000ACF1010C0CEBCC0C4FEA4C0C0CF1050C4D
:100B9000DFF8F89019F80CC048EA0C2CA3F800C054
:100BA00090F800C0ACF1010C0CEBCC0C4FEA4C0CF3
:100BB0000CF1080CC84618F80C8090F800C0ACF195
:100BC000010C0CEBCC0C4FEA4C0C0CF1070C19F897
:100BD0000CC048EA0C2CA4F800C090F800C0ACF19E
:100BE000010C0CEBCC0C4FEA4C0C0CF10A0CC84677
:100BF00018F80C8090F800C0ACF1010C0CEBCC0C98
:100C00004FEA4C0C0CF1090C19F80CC048EA0C2CFA
:100C1000A5F800C090F800C0ACF1010C0CEBCC0CB6
:100C20004FEA4C0C0CF10C0CC84618F80C8090F8EC
:100C300000C0ACF1010C0CEBCC0C4FEA4C0C0CF1ED
:100C40000B0C19F80CC048EA0C2CA6F800C090F860
:100C500000C0ACF1010C0CEBCC0C4FEA4C0C0CF1CD
:100C60000E0CC84618F80C8090F800C0ACF1010CCE
:100C70000CEBCC0C4FEA4C0C0CF10D0C19F80CC021
:100C800048EA0C2CA7F800C0BDE8F0831A00002049
:100C900010B5012000F09CFB002000F099FB10BD76
:100CA000014908607047000000860D4208B5002227
:100CB0000092044A0092009A02440092009A116045
:100CC00008BD0000006C004070B50246CB78137080
:100CD000042000BF0AE00D5C431E1478641E122637
:100CE00006FB0433034CE554431CD8B21028F2DB56
:100CF00070BD00001A00002000BFFEE770472DE91C
:100D0000F041024600250026002000230024002791
:100D100091F803C00CF00F0591F803C00CF0100C13
:100D2000BCF1000F03D091F802C04CEA050591F820
:100D300000C0BCF1000F31D0146800202BE04FF050
:100D4000010C0CFA00F3B1F800C00CEA03069E4255
:100D500020D183004FF00F0C0CFA03F7BC4305FAC7
:100D600003FC4CEA040491F803C0BCF1280F06D13F
:100D70004FF0010C0CFA00FCC2F814C00AE091F824
:100D800003C0BCF1480F05D14FF0010C0CFA00FC78
:100D9000C2F810C0401C0828D1D31460B1F800C0BC
:100DA000BCF1FF0F34DD546800202EE000F1080C88
:100DB0004FF0010808FA0CF3B1F800C00CEA030682
:100DC0009E4221D183004FF00F0C0CFA03F7BC4375
:100DD00005FA03FC4CEA040491F803C0BCF1280FA7
:100DE00005D100F1080C08FA0CF8C2F8148091F84B
:100DF00003C0BCF1480F07D100F1080C4FF0010807
:100E000008FA0CF8C2F81080401C0828CED35460B1
:100E1000BDE8F081416170470161704708B501216B
:100E2000112000F0B5FA012000F09CFA002000F03B
:100E300083FB0020FFF734FF4FF46040ADF8000063
:100E400002208DF8020010208DF803006946064844
:100E5000FFF755FF002000F085FA4FF4604102488B
:100E6000FFF7DAFF08BD00000010014010B504468E
:100E700001200D4908600D49C1F8B801204600F075
:100E800017F800200849091F0860022003F082F9C2
:100E900001200649C1F8B801022003F07BF90020C7
:100EA0000149091F086010BDBC0122420000224216
:100EB00070B50446002500BF18E004F0800018B1AA
:100EC00001200C49086002E000200A490860002067
:100ED0000849083108600A2003F03CF9012006495E
:100EE000C1F8BC016006040E681CC5B2082DE4DB25
:100EF00070BD0000B40122420000224200BFFEE7A4
:100F00000146CA1701EB92729210A1EB820292B9CC
:100F1000642091FBF0F200FB121050B94FF4C8703E
:100F200091FBF0F200FB121008B90120704700207D
:100F3000FCE70120FAE70020F8E700BFFEE7704772
:100F400070B5002100230F22C47804B3154C246827
:100F500004F4E064C4F5E064210AC1F10403CA406A
:100F6000447804FA03F184781440214309010E4CBB
:100F70000678A155047804F01F050124AC400578DB
:100F80006D11AD0005F1E025C5F8004109E00478D8
:100F900004F01F050124AC40044D0678761145F895
:100FA000264070BD0CED00E000E400E080E100E0D0
:100FB00002490143024A1160704700000000FA052F
:100FC0000CED00E070B55648806B5549C968884201
:100FD00000DA70BD524948684FF07E51FFF702F9C0
:100FE00006464F4801683046FFF7E8FB0BD24D49F3
:100FF000097801F0FB014B4A11700846FFF736FFF4
:10100000022049490870464908684FF07E51FFF7B1
:10101000E9F80646424841683046FFF7CFFB0BD25D
:101020004049097841F004013E4A11700846FFF733
:101030001DFF01203C490870394A51681068FFF7CC
:10104000C7FB07D2364A51681068FFF71DF93449CB
:10105000886106E0324A11685068FFF715F9304997
:1010600088612F4A91699068FFF714F92C498862CA
:101070000A469169106AFFF7B5F8294908620A46DD
:10108000D1699069FFF700F905462548016A2748AC
:101090000068FFF7FFF822494862294624480068A3
:1010A000FFF7F8F81E49C862C86A0021FFF786FBFF
:1010B00006D21B48C16A0020FFF7E6F81849C8624B
:1010C000174A516A906AFFF78DF806461448C16ABC
:1010D0003046FFF787F804461149C86BFFF7D2FA8C
:1010E00006462146FFF76AFB06D20D49C86BFFF79B
:1010F000C9FA0B4948630BE000212046FFF75EFB6D
:1011000004D80748006B0649486301E0044844637B
:10111000034880690249C8610020886300BF58E71E
:10112000680300206C01002074010020CC00002026
:10113000D00000200648074988604FF4FA70C86064
:10114000C820C8634FF07E50086300208863704752
:1011500000002A436803002030B589B005460C46DC
:101160000121C80200F014F90121042000F010F957
:1011700018208DF823004FF48070ADF82000032074
:101180008DF8220008A91B48FFF7B9FD0020ADF833
:101190001A00ADF81600ADF81850ADF814408DF8EF
:1011A0001C0005A9144802F001F801A801F0EDFFA8
:1011B0006020ADF804000020ADF80C000120ADF86F
:1011C00006000020ADF80A0001A90B4801F090FECE
:1011D0000121094801F063FE0821074801F0D4FE0F
:1011E0000121054801F040FE0121034801F04BFEBA
:1011F00009B030BD00080140002C014030B589B075
:1012000005460C460121C80200F0C2F80121042065
:1012100000F0BEF818208DF823004FF40060ADF800
:10122000200003208DF8220008A91B48FFF767FD66
:101230000020ADF81A00ADF81600ADF81850ADF862
:1012400014408DF81C0005A9144801F0AFFF01A857
:1012500001F09BFF6020ADF804000020ADF80C0009
:101260000120ADF806000020ADF80A0001A90B48E6
:1012700001F040FF0121094801F011FE0821074853
:1012800001F076FF0121054801F0EEFD0121034840
:1012900001F0F9FD09B030BD00080140002C01400B
:1012A00030B589B005460C460121084600F060F8CB
:1012B0000121042000F06CF818208DF82300022092
:1012C000ADF8200003208DF8220008A91648FFF78A
:1012D00016FD0020ADF81A00ADF81600ADF8185054
:1012E000ADF814408DF81C0005A94FF0804001F0C6
:1012F0005DFF01A801F049FF6020ADF80400002067
:10130000ADF80C000120ADF806000020ADF80A0091
:1013100001A94FF0804001F041FE0121880701F052
:10132000B2FD09B030BD00000008014010B5044610
:101330002146024801F033FF10BD0000002C01409F
:1013400010B5044621464FF0804001F02AFF10BD41
:1013500010B504462146024801F025FF10BD0000EB
:10136000002C0140014908627047000000000E4255
:1013700029B1064AD2690243044BDA6104E0034A08
:10138000D2698243014BDA617047000000100240CD
:1013900029B1064A92690243044B9A6104E0034A68
:1013A00092698243014B9A6170470000001002402D
:1013B00029B1064AD2680243044BDA6004E0034ACA
:1013C000D2688243014BDA6070470000001002408F
:1013D00001490860704700004004424230B50021D6
:1013E0000022002400232D4D6D6805F00C0121B171
:1013F000042905D0082923D105E0294D056022E004
:10140000274D05601FE0254D6D6805F47012234DD2
:101410006D6805F48034022505EB92421CB9214D1C
:10142000554305600BE01D4D6D6805F400351DB199
:101430001C4D5543056002E0194D5543056002E01F
:10144000174D056000BF00BF144D6D6805F0F00139
:101450000909154D6B5C0568DD4045600F4D6D68F1
:1014600005F4E061090A104D6B5C4568DD4085605C
:101470000A4D6D6805F46051C90A0B4D6B5C4568F7
:10148000DD40C560054D6D6805F44041890B074D91
:101490006B5CC568B5FBF3F5056130BD001002401B
:1014A00000127A0000093D00DA000020EA00002066
:1014B00010B501460022002300204A11012A02D162
:1014C000094C236806E0022A02D1074C236A01E096
:1014D000054C636A01F01F02012494401C400CB1CA
:1014E000012000E0002010BD0010024011490968F1
:1014F00021F480310F4A11601146096821F48021DE
:101500001160B0F5803F03D0B0F5802F0ED106E01A
:101510000849096841F48031064A116007E005492D
:10152000096841F4A021034A116000E000BF00BF38
:10153000704700000010024000210B4A11700A4A57
:10154000203A82F82010012802D0042808D103E0B4
:101550000121054A117004E00521034A117000E0E1
:1015600000BF00BF70470000201002400149086022
:10157000704700003C0442420249096A0143014AA3
:10158000116270470010024010B586B0044600F0AA
:10159000ABFD20213348FFF73DFC40213148FFF7E8
:1015A0003BFC01210C20FFF7F3FE01218803FFF72C
:1015B000EFFE4FF40060ADF8140010208DF8170016
:1015C00003208DF8160005A92648FFF798FB4FF475
:1015D0000070ADF8140018208DF8170005A92248F6
:1015E000FFF78DFB4FF48060ADF8140004208DF8F8
:1015F000170005A91C48FFF782FB01218803FFF7AC
:10160000D7FE00214FF48040FFF7D2FE0194002066
:10161000ADF80800ADF80A00ADF80C00ADF8100008
:101620000C20ADF80E0001A9104801F085FF25201F
:101630008DF8000000208DF8010001208DF80300D6
:101640006846FFF77DFC012240F22551074801F072
:101650004EFF0121054801F007FF00200449086002
:1016600006B010BD000C01400008014000380140E8
:10167000AC81214270B505460E4601200E49086036
:1016800000240CE000BF40210C4801F0F9FE0028C6
:10169000F9D0295D094801F0C0FF601CC4B2B44212
:1016A000F0DB00BF4021054801F0EAFE0028F9D038
:1016B00000200149086070BDAC8121420038014022
:1016C00010B50120A4490860A4480068B0F5FA7F6D
:1016D00007DCA348C078A3490870A1480079A24953
:1016E0000870A2480068B0F57A7F07DC9C48407912
:1016F0009F4908709A4880799E49087099480078F7
:101700009D49C870984800780871994800784871D8
:1017100098480078887199480078401E00EBC00016
:1017200040000A309649095C94480078401E00EB5E
:10173000C00040000930924A105C41EA0020914903
:1017400008808E480078401E00EBC00040000C303E
:101750001146095C89480078401E00EBC00040003B
:101760000B30105C41EA00208749088083480078EC
:10177000401E00EBC00040000E301146095C7F485F
:101780000078401E00EBC00040000D30105C41EAC4
:1017900000207E4908807B480088B0F57A7F15DC00
:1017A00076480078401E00EBC0004000093011462A
:1017B000085C7749087071480078401E00EBC00053
:1017C00040000A301146085C724908706E48008873
:1017D000B0F57A7F15DC69480078401E00EBC00048
:1017E00040000B306649085C6B490870634800781C
:1017F000401E00EBC00040000C306149085C6749A6
:10180000087062480088B0F57A7F15DC5B48007884
:10181000401E00EBC00040000D305949085C604993
:10182000087056480078401E00EBC00040000E30A3
:101830005349085C5B490870554800784E49C871A7
:101840005448007808725448007848725348007829
:10185000887253480078C87252480078087352481A
:10186000006841F28831884207DC3D48C07C4F491E
:1018700008703B48007D4E4908704C4800783E494E
:1018800048734B48007888733C480078072802DA90
:101890003A480078C87339480078401E00EBC00011
:1018A0004000C01C3649085C182809DA3348007823
:1018B000401E00EBC0004000C01C085C2E490874AC
:1018C0002E480078401E00EBC0004000001D2C494F
:1018D000085C3C2809DA29480078401E00EBC0006B
:1018E0004000001D085C24494874324800781828DC
:1018F00003DA30480078204988742F4800783C2863
:1019000003DA2D4800781C49C8742C4800781A491D
:1019100008752B48007848752A4800788875002497
:101920000DE000BF4021284801F0AAFD0028F9D0B1
:101930001148015D244801F070FE601CC4B21B2CEC
:10194000EFDB00BF4021204801F09AFD0028F9D0CC
:1019500000200149086010BDAC81214294010020A3
:10196000DC020020A3000020A40000209801002039
:10197000A5000020A6000020860000207A0100209B
:101980001A000020AA000020AE000020AC000020B9
:10199000B0000020B1000020B4000020B5000020FD
:1019A000B2000020B30000209C010020A70000200E
:1019B000A8000020720100207301002074010020A3
:1019C0007501002076010020003801401CB519A1E6
:1019D00003C9CDE9000101201849086018480078C2
:1019E0008DF8030016480078401C15490870084619
:1019F0000078062801DD0120087000240DE000BFFA
:101A00004021104801F03CFD0028F9D01DF80410D9
:101A10000C4801F002FE601CC4B2082CEFDB00BFD2
:101A20004021084801F02CFD0028F9D0002003498E
:101A300008601CBDEEB50100FFFCFFFFAC81214238
:101A40006D01002000380140024909888143014AA4
:101A500011807047042800400348008840F01000BF
:101A600001490880704700000428004003480088AE
:101A70004FF6EF7108400149088070470428004084
:101A80002DE9F04106460F464FF0000800240025DE
:101A900000F082F880463C48B8FBF0F43B480088F0
:101AA000A0423CD039490C8040F2B27510E0284683
:101AB000FFF726FA40B1B4F5B77F02D3A4F5B774A7
:101AC00004E0681C85B206E0A4F26D14681C85B2BF
:101AD000B4F5B67FEBD800BF2D488580002516E011
:101AE0002B498888FFF70CFA30B1012D04D11D2C49
:101AF00001D31D3C09E00CE02648405DA04203D81C
:101B00002448405D241A00E003E0681C85B21C2CC8
:101B1000E6D200BF681C1E498871601CC8711A4853
:101B2000B8FBF0F100FB11844FF46160B4FBF0F0FE
:101B3000174908704FF46160B4FBF0F100FB1140ED
:101B40003C21B0FBF1F0124948704FF46160B4FBE6
:101B5000F0F100FB11403C21B0FBF1F201FB12005F
:101B60000B4988700B46DA799979988800F030F83B
:101B70000749087208460078307008464078387087
:101B80000020BDE8F081000080510100BC00002071
:101B90005C03002018670008002103480188001F2B
:101BA000008841EA004070471C28004001460020A0
:101BB000064A12880A40D0B2044A121F12880A400C
:101BC00012B108B1012000E0002070470428004055
:101BD000F0B503460C461546642093FBF0F0C6B200
:101BE000642093FBF0F700FB1730C1B2132E02DD27
:101BF00001F16400C1B20846CF1701EB977701EB02
:101C0000A707BAB2072092FBF0F700FB172082B2B9
:101C10005719601EDFF82CC01CF80000384482B24F
:101C2000CF1701EB9777BF10A1EB87071FB9032CE4
:101C300001DA501E82B2072092FBF0F700FB17205A
:101C4000C0B2F0BD0C6700080EB50120FFF7AEFF73
:101C500098B11A491A48FFF713FF1A4880781949B2
:101C60004978184A1278CDE9002102901548C379C5
:101C70008279818814A001F0FBFD0220FFF796FF16
:101C8000B0B10220FFF7E0FE0C490D48FFF7F8FE67
:101C90000C4880780B4949780A4A1278CDE900212E
:101CA00002900848C379827981880FA001F0E0FD95
:101CB0000520FFF7C9FE00F041F90EBDBB00002072
:101CC000BA0000205C0300205254432054696D6523
:101CD0003A25642D25642D25642025643A25643A2F
:101CE00025640D0A00000000416C61726D2054698A
:101CF0006D653A25642D25642D25642025643A25DB
:101D0000643A25640A00000029B1064A1288024399
:101D1000044B1A8004E0034A12888243014B1A8064
:101D200070470000002800401CB52DA001F0A0FD68
:101D3000002401214FF0C050FFF71AFB0120FFF7EC
:101D400011FBFEF7A5FF4FF48030FFF7CFFB04E057
:101D5000601CC4B20A2002F0FDF93120FFF7A8FB95
:101D600008B9FA2CF4DBFA2C01DB01201CBD21A000
:101D700001F07EFD4FF44070FFF7FEFB20A001F064
:101D800077FD0120FFF7F2FB00F0D8F800F0E0F853
:101D900001210846FFF7B8FF00F0D0F8FFF75CFE1E
:101DA0004FF2244000F0BAF800F0C8F8002000908C
:101DB000034601220921019040F2E77000F03CF84F
:101DC000FFF754FE45F250010420FEF76FFF00F0CC
:101DD00025F810491048FFF753FE0020C6E7000021
:101DE0007274635F696E69742073746172740D0A32
:101DF000000000007274635F696E6974200D0A0050
:101E00004853452069732074696D65736F757263FB
:101E1000650D0A00BB000020BA00002008B50320B1
:101E20008DF8000001208DF801008DF80300684650
:101E3000FFF786F808BD00002DE9F05F06460F4663
:101E400090469946DDE90AAB002440F2B270864222
:101E500003DB40F63300864202DD0120BDE8F09F3F
:101E600040F2B2750AE02846FFF74AF810B1204860
:101E7000044401E01F480444681C85B2B542F2DB0B
:101E8000781EC7B2002510E01B48405D40F2A32138
:101E9000484304EBC0143046FFF732F818B1012D67
:101EA00001D116480444681C85B2BD42ECDBA8F1A0
:101EB000010040F2A321484304EBC014C9EB4910D0
:101EC000C0EB092004EB0014CAEB0A1004EB8004F9
:101ED0005C4401214FF0C050FFF74AFA0120FFF7A0
:101EE00041FA204600F00CF800F028F80020B5E791
:101EF0000085E2018033E10118670008805101008C
:101F000000B50246FFF7A8FD100C03490880091D23
:101F10000A80FFF7ABFD00BD1828004000B502465F
:101F2000FFF79AFDC2F3034003490880091D0A80A8
:101F3000FFF79CFD00BD00000828004000BF0348DB
:101F4000008800F020000028F9D0704704280040E5
:101F5000074800884FF6F77108400549088000BF20
:101F60000348008800F008000028F9D070470000FE
:101F7000042800402DE9FC4705460E4617469846C2
:101F8000DDE90A9A002401214FF0C050FFF7F0F973
:101F90000120FFF7E7F9FEF77BFE4FF48030FFF7F3
:101FA000A5FA04E0601CC4B20A2002F0D3F8312084
:101FB000FFF77EFA08B9FA2CF4DBFA2C02DB0120D9
:101FC000BDE8FC874FF44070FFF7D6FA0120FFF719
:101FD000CDFAFFF7B3FFFFF7BBFF01210846FFF77C
:101FE00093FEFFF7ABFFFFF737FD4FF22440FFF7FB
:101FF00095FFFFF7A3FF43463A4631462846CDE911
:10200000009AFFF719FFFFF731FD45F25001042058
:10201000FEF74CFEFFF702FF02490348FFF730FDD1
:102020000020CDE7BB000020BA00002070B50546B7
:10203000002400BF05E00448015D04A001F018FC85
:10204000641CAC42F7DB70BDDC0200202578200068
:1020500010B502460020104604E043180B4CE35C28
:102060002354401CC1F140038342F6DCC1F140001F
:1020700003E00023054C2354401C4028F9DB044BAB
:102080001B785B1A024C237010BD0000DC0200209C
:10209000B80000200146002003E00022024B1A5441
:1020A000401C8842F9DB7047DC02002010B56C222E
:1020B00000210A4801F004FB6D230022074908486B
:1020C00002F03BF8002405E00448015D05A001F0A2
:1020D000CFFB641C6C2CF7DB10BD0000F00100206E
:1020E0005C0200202578200008B501210820FFF7B8
:1020F0004FF9E020ADF8000010208DF80300032018
:102100008DF8020069460448FEF7F9FD8021024877
:10211000FEF780FE08BD0000000C014000B587B04E
:1021200001210420FFF734F901210803FFF730F9FA
:10213000E020ADF8180018208DF81B0003208DF862
:102140001A0006A91748FEF7DAFDE0211548FEF748
:1021500063FE0020ADF804004FF48270ADF8060075
:102160000020ADF808000220ADF80A000120ADF80B
:102170000C004002ADF80E003820ADF81000002031
:10218000ADF812000720ADF8140001A9064800F0D0
:1021900067F80121044800F049F8FF2000F006F834
:1021A00007B000BD000801400030014070B5054691
:1021B000002405E0601CC4B2C82C01DD002070BD05
:1021C00002210E4800F03EF80028F3D029460B48C3
:1021D00000F044F8002405E0601CC4B2C82C01DD06
:1021E0000020ECE70121054800F02CF80028F3D08E
:1021F000024800F030F8C0B2E1E7000000300140D2
:1022000010B50446074800884FF6C77108400549D5
:10221000088008460088204308800121024800F019
:1022200005F810BD003800400030014021B102889F
:1022300042F04002028004E002884FF6BF731A4069
:10224000028070470246002013890B400BB1012029
:1022500000E00020704701468889704781817047FF
:1022600010B50022028802F441520B884C882343A7
:102270008C882343CC8823430C8923434C892343F4
:102280008C892343CC8923431A430280838B4FF2EA
:10229000FF74234083830B8A038210BD9CB089E3C3
:1022A000FFF704FF02F004FFFA490870FA480278C9
:1022B000FA480178FAA001F0DBFAFC48FC49FD4A33
:1022C000FD4BCDE90032CDE90210FC4BFC4AFD4943
:1022D000F048FEF725FCEF480178FBA001F0C8FAB2
:1022E0000821FE48FFF7C6F9FDA001F0C1FA4FF43E
:1022F0007A7001F073FF8020FFF798FEFFF766FB0E
:102300004FF47A7001F06AFF8020FFF78FFED6E26B
:10231000F7A001F0ADFAFA480078012872D1F84828
:1023200040780328FAD1F648C078F6490860F448A6
:102330000079096840EA0120F2490860F0484079D4
:10234000F1490860EE488079096840EA0120EE49C9
:102350000860EB48C07CED490860E948007D0968E9
:1023600040EA0120E9490860E74800680A2190FB3B
:10237000F1F201FB1204E448006890FBF1F5E1483A
:10238000006890FBF1F201FB1206DE48006890FB4A
:10239000F1F7DE4800682B4632463946CDE9004069
:1023A000DBA001F065FAC54800881438D5490968F2
:1023B000884214DCD3480168C04800881430814248
:1023C0000DDCBD4800886438CF490968884206DCC6
:1023D000CD480168B84800886430814213DDD74891
:1023E000008840F2622188420DDDD549097841F02C
:1023F0000101D34A11700846FEF738FD0120D1498A
:1024000008700CE0C1E1CE49097801F0FE01CC4A28
:1024100011700846FEF72AFD0020CA490870B94825
:102420000068B0F5167F7DDAB648006810F11E0F1F
:1024300078DDC5480068B3490968401AC349086097
:1024400008460068002803DA084600684042086031
:10245000BE480068032803DBBB480068002861D140
:1024600096480088FEF728F906460022B84BFEF78A
:102470009AF80446FEF786F9B6490860A148006854
:10248000FEF709F906460022B14BFEF78CF8044628
:10249000FEF778F9AF494860FEF794FDAD49C86B87
:1024A000FEF7F0F80646AB49486BAB49FDF7F2FE84
:1024B00007463146FDF720FF05464FF07E51FDF7F8
:1024C000E3FE0446FEF705F9A449086008460088C3
:1024D00081B2A34800F067FEA0480068FEF7ECF860
:1024E000804600229F4BFEF75EF804460D46994950
:1024F000C86AFEF71BF906460F469649486AFEF77A
:1025000015F982468B469349886AFEF70FF9CDE9A3
:102510001A0195480068FEF709F9CDE918019348BA
:10252000006800E03DE0FEF701F9CDE916018949B8
:102530008868FEF7FBF8CDE91401864908688C49E4
:10254000FDF7A8FE8046FEF7F1F8CDE90CABCDE92A
:102550000E67CDE91045CDE91201DDE91A01CDE99B
:102560000A01DDE91801CDE90801DDE91601CDE92F
:102570000601DDE91401CDE90401DDE91201CDE92F
:102580000201764800680090604803685E4802686F
:102590005C480168774801F06BF95A4800686A495D
:1025A000086059480168444800883230814214DD8F
:1025B0006349097841F00801614A11700846FEF745
:1025C00055FC5F49097801F0EF015D4A117008463A
:1025D000FEF74CFC01206849087037480088323803
:1025E00049490968884214DD5549097841F01001CC
:1025F000534A11700846FEF739FC5149097801F039
:10260000F7014F4A11700846FEF730FC02205A4984
:10261000087059480078012811D13B4800682649C4
:10262000098888420BDC4649097801F0E701444AF1
:1026300011700846FEF71AFC00204F4908704E48FA
:102640000078022811D1304800681B490988884267
:102650000BDB3B49097801F0E701394A1170084664
:10266000FEF704FC00204449087044A001F000F982
:10267000FFF726F81720FFF70DFD17210020FFF7C1
:10268000E7FC3FA001F0F4F88020FFF7CFFC3CA06E
:1026900078E000007A010020730100207201002020
:1026A0002564202025640D0A00000000840100201C
:1026B00082010020800100207E0100207C0100209A
:1026C000870100208601002063757272656E742098
:1026D00073746167653A2025640D0A008B01002040
:1026E00073656E642066696E6973680D0A00000088
:1026F000656E746572207768696C650D0A0000006C
:10270000DC02002094010020980100209C010020A0
:102710006E6F775F74656D3D25642E2564A1E62C90
:102720006E6F775F68756D3D25642E2564252520C5
:102730002C636F323D25640D0A00000078010020F3
:102740006C01002076010020A40100206801002017
:1027500000002440680300200000C843B0010020AE
:102760000008004000F07840D0000020CC0000209D
:102770000000204170670008750100202121210020
:102780000D0A000001F074F899E08B480078EE28FB
:1027900025D189484078B62821D1874880780328F8
:1027A0001DD1854A85498648FEF77EF985A001F04E
:1027B0005FF80B20FFF76EFC88A001F059F80B21A1
:1027C0000020FFF745FCAFF2480001F051F88020EF
:1027D000FFF72CFCAFF2580001F04AF86FE07648A2
:1027E0000078EE282FD174484078B6282BD1724853
:1027F0008078042827D17048C0787949087079A07A
:1028000001F036F8002000900346012209210190D2
:1028100040F2E770FFF7AEFB714800787849087026
:102820000820FFF737FC6DA001F022F808210020F6
:10283000FFF70EFCAFF2B80001F01AF8AFF2C000DB
:1028400001F016F83BE05C480078EE2825D15A48A4
:102850004078B62821D15848807801281DD15649A2
:102860005748FEF731FA5648017866A001F000F8A3
:1028700000F0F0FF1420FFF70DFC58A000F0F8FF67
:1028800014210020FFF7E4FBAFF20C1000F0F0FF82
:10289000AFF2141000F0ECFF11E060A000F0E8FFD0
:1028A00001210020FFF7D4FB4CA000F0E1FFAFF2C4
:1028B000301000F0DDFFAFF2381000F0D9FF3E48D5
:1028C000007800287FF424AD3B4840780028F9D1F7
:1028D000394880780028F5D13748C0780028F1D1F0
:1028E000354800790028EDD1524803685248026803
:1028F0005248016852A000F0BBFF56480078564984
:102900000978CDE9001055480378554802785548B4
:102910000178554800F0ACFF54A000F0A9FF5648DC
:102920000088B0F57A7F42DC54480088B0F57A7FA1
:102930003DDC51480088FDF7BFFE82460022504B27
:10294000FDF731FE804600224E4BFDF7BAFD0646EC
:1029500000224D4BFDF70EFD0446FDF7CEFE80B282
:102960001B90FEF7E3FC45480088FDF7A5FE0646F0
:102970000022434BFDF717FE80460022414BFDF736
:10298000A0FD04460022404BFDF7F4FC8246FDF713
:10299000B4FE80B21B90FEF7D3FC374801883BA001
:1029A00000F066FF354801883BA000F061FF002081
:1029B0003C49087074E40000DC0200207001002033
:1029C0006E010020423620303320636D643A20626D
:1029D000617463682073796E630D0A00200D0A002C
:1029E00088010020423620303420636D643A206331
:1029F00068616E67652073746167650D0A00000089
:102A00007A010020423620303120636D643A20671D
:102A10006574206F6E652025640D0A0070726576FE
:102A2000696F7573206172726179206375740D0A24
:102A3000000000009C01002098010020940100206B
:102A400025642020202025642020202020202564AB
:102A50000D0A00007601002075010020740100209D
:102A60007301002072010020246700086C65642156
:102A700021210D0A000000008001002082010020B9
:102A80000000594000000C4000003C407265643D6D
:102A900025640D0A0000000062756C653D25640D1B
:102AA0000A000000B800002010B500F001F810BDC9
:102AB0000CB50020019000903348006840F480304D
:102AC0003149086000BF3048006800F400300090D1
:102AD0000198401C0190009818B90198B0F5A06FBA
:102AE000F1D12948006800F4003010B101200090B5
:102AF00001E0002000900098012843D1234800689D
:102B000040F01000214908600846006820F00300EA
:102B100008600846006840F0020008601A484068F3
:102B2000194948600846406848600846406840F4D3
:102B3000806048600846406820F47C104860084681
:102B4000406840F4E81048600846006840F0807033
:102B5000086000BF0C48006800F000700028F9D041
:102B60000948406820F0030007494860084640686B
:102B700040F00200486000BF0348406800F00C00CD
:102B80000828F9D10CBD00000010024000200240CE
:102B9000042808D14FF0E021096941F004014FF009
:102BA000E022116107E04FF0E021096921F0040102
:102BB0004FF0E0221161704710B503F001FB0128CE
:102BC00001D002F01FFF10BD70B505460420FFF7CD
:102BD000DFFF104800681049B0FBF1F00F490870A2
:102BE0000C4800680C49B0FBF1F44FF47A70444390
:102BF00001200B4908804FF0E020006940F00200FE
:102C00004FF0E021086108464461006940F001008E
:102C1000086170BD0000002040420F00D400002079
:102C2000D600002010B51348006840F0010011499B
:102C3000086008464068104908400E494860084648
:102C400000680E4908400B4908600846006820F4F7
:102C5000802008600846406820F4FE0048604FF479
:102C60001F008860FFF720FF4FF0006004490860F4
:102C700010BD0000001002400000FFF8FFFFF6FE4C
:102C800008ED00E010B50121064800F017F940B149
:102C90000548806B401C044988630121014800F00D
:102CA000EFF810BD00040040680300201FB50121AB
:102CB0000220FEF75DFB1D208DF80C0003208DF82F
:102CC0000D0001208DF80F0003A8FEF739F94FF42D
:102CD0007A70ADF804004720ADF800000020ADF890
:102CE00002006946084800F061FA012211460648D0
:102CF00000F0F5F80121044800F0C2F80121024873
:102D000000F0C1F81FBD0000000400402DE9F04FA5
:102D100087B001212F4800F0D1F8002857D00121B9
:102D20002C4800F0ADF82C480088401C2A49088047
:102D30002A480088B0F57A7F40DC284800880028BF
:102D40003CDD27480078462833DC25480078FEF72C
:102D5000FFFA22480088FDF7AFFC80460022214B95
:102D6000FDF721FC4FF066321F4BCDE90001FDF766
:102D7000A8FB064600221D4BFDF7FCFA0446002284
:102D80001B4BFDF710FC82468B4615480078FDF77B
:102D900093FC52465B46CDE90201FDF7EBFACDE923
:102DA0000401FDF7AAFC0E49087012A000F060FDB6
:102DB00004E000200A490870FEF7CAFA07480088B4
:102DC00028B90020FEF7C4FA0DA000F051FD07B0AD
:102DD000BDE8F08F00080040780100208401002049
:102DE00064010020000059406666064000003E4035
:102DF0000000184077686974652070776D0D0A00CF
:102E000077686974652069732030212121000000F2
:102E10007FB505460C4601210420FEF7A9FAADF85E
:102E20000850ADF804400020ADF80A00ADF80600E7
:102E300001A90C4800F0BAF901221146094800F036
:102E40004EF81E208DF8000002208DF801000120B0
:102E50008DF803006846FEF773F80121014800F081
:102E600012F87FBD0008004021B1028842F08002C4
:102E7000028004E002884FF67F731A400280704798
:102E8000CA430282704721B1028842F001020280E7
:102E900004E002884FF6FE731A400280704731B199
:102EA000B0F8442042F40042A0F8442005E0B0F815
:102EB0004420C2F30E02A0F84420704730B5024609
:102EC000002000230024158A05EA0103958905EAFC
:102ED000010413B10CB1012000E0002030BD1AB193
:102EE00083890B43838102E083898B43838170470D
:102EF00070B5002400220023058C4FF6FE76354085
:102F00000584028C8388048B4FF68F752C40B51E88
:102F10002C400D882C43751E2A400D892A434D886C
:102F20002A43144DA8420BD0134DA84208D0134D8C
:102F3000A84205D0124DA84202D0124DA84213D18A
:102F40004FF6F7752A404D892A434FF6FB752A4004
:102F50008D882A434FF6FF652B404FF6FF552B40D7
:102F60008D892B43CD892B4383800483CD8885862F
:102F7000028470BD002C014000340140004001403B
:102F800000440140004801400A460021018B4FF6F1
:102F9000F7731940114301837047000070B5002496
:102FA00000220023058C4FF6EF7635400584028C15
:102FB0008388048B48F6FF752C404FF6FF452C4064
:102FC0000D884FF6FF7606EA05252C434FF6DF7590
:102FD0002A400D8906EA05152A434D8806EA05159B
:102FE0002A43154DA84202D0144DA8421DD14FF6D8
:102FF0007F752A404D894FF6FF7606EA05152A436C
:103000004FF6BF752A408D8806EA05152A434FF60C
:10301000FF352B404FF2FF752B408D8906EA850561
:103020002B43CD8906EA85052B4383800483CD8815
:103030000587028470BD0000002C0140003401406F
:1030400070B5002400220023058C4FF6FF66354042
:103050000584028C8388848B4FF68F752C404FF645
:10306000FC752C400D882C434FF6FF552A400D89E6
:103070004FF6FF7606EA05252A434D8806EA052520
:103080002A43154DA84202D0144DA8421DD14FF23B
:10309000FF752A404D894FF6FF7606EA05252A433B
:1030A0004FF6FF352A408D8806EA05252A434EF65D
:1030B000FF752B404DF6FF752B408D8906EA0515EF
:1030C0002B43CD8906EA05152B4383808483CD8865
:1030D0008587028470BD0000002C0140003401404F
:1030E0000A460021818B4FF6F77319401143818303
:1030F0007047000070B5002200230024058C4EF6B6
:10310000FF7635400584038C8488828B48F6FF75F2
:103110002A404FF6FF452A400D884FF6FF7606EA13
:1031200005252A434DF6FF752B400D8906EA053526
:103130002B434D8806EA05352B430B4DA84202D0A0
:103140000A4DA84208D14BF6FF752C408D894FF6E9
:10315000FF7606EA85152C4384808283CD88A0F80B
:103160004050038470BD0000002C01400034014039
:103170000A460021818B4FF2FF7319404FF6FF730F
:1031800003EA0223194381837047002101804180B3
:103190008180C180018141818181C18170478186A7
:1031A000704701877047A0F84010704700220288DE
:1031B0001D4B98420ED01D4B98420BD0B0F1804F62
:1031C00008D01B4B984205D01A4B984202D01A4B9C
:1031D000984204D14FF68F731A404B881A43174B0D
:1031E000984207D0164B984204D04FF6FF431A403E
:1031F000CB881A4302808B8883850B8803850A4B12
:1032000098420BD0094B984208D00E4B984205D0FB
:103210000D4B984202D00D4B984201D10B7A038698
:103220000123838270470000002C014000340140DC
:103230000004004000080040000C00400010004066
:10324000001400400040014000440140004801409B
:1032500030B589B005460C4601210920FEF798F8E3
:103260000120ADF8200018208DF8230003208DF8F0
:10327000220008A91648FDF742FD01210220FEF7B1
:1032800077F8A8B2ADF81800A0B2ADF8140000208D
:10329000ADF81A00ADF8160005A90E48FFF786FF35
:1032A0007020ADF804000120ADF806000220ADF852
:1032B0000C0001A90748FFF7C3FE08210548FFF7E6
:1032C0000FFF01210348FFF7DEFD09B030BD00000C
:1032D000000C01400004004010B540F225510B489D
:1032E00000F0DBF880B1094800F092F9C4B2084858
:1032F0000078402808DA074805490978445404480A
:103300000078401C0249087010BD000000380140E0
:10331000B8000020DC02002010B540F225511D4805
:1033200000F0BBF810B31B4800F072F9C4B21A48A1
:10333000008800F40040C8B91748008800F48040B5
:1033400060B10A2C03D000201349088020E0124805
:10335000008840F400401049088019E00D2C06D187
:103360000D48008840F480400B49088010E00A486E
:103370000088C0F30D0009490C5407480088401C20
:103380000549088008460088FE2801DD00200880E5
:1033900010BD000000440040D8000020AC03002015
:1033A00010B586B0044601214804FDF7E1FF012174
:1033B0000C20FDF7EDFF4FF40070ADF81400032072
:1033C0008DF8160010208DF8170005A92248FDF78A
:1033D00096FC0420ADF8140003208DF81600182088
:1033E0008DF8170005A91D48FDF789FC0820ADF8E8
:1033F000140004208DF8170005A91848FDF77FFC7C
:1034000026208DF8000004208DF8010001208DF8A1
:1034100003006846FDF794FD01940020ADF8080014
:10342000ADF80A00ADF80C00ADF810000C20ADF8B6
:103430000E0001A90A4800F07FF8012240F2255150
:10344000074800F054F80121054800F00DF800206D
:103450000449086006B010BD000C0140000801409E
:1034600000440040A481214221B1828942F40052EB
:10347000828104E082894DF6FF731A408281704791
:1034800002460020B1F5007F00D100BF13880B4039
:103490000BB1012000E00020704770B50246002407
:1034A00000230025002040F66A16B14200D100BF7B
:1034B000C1F3421501F01F03012606FA03F3012DA3
:1034C00002D19689334006E0022D02D1168A33409C
:1034D00001E0968A33400C12012606FA04F416889D
:1034E000344013B10CB1012000E0002070BDF0B5F4
:1034F0000346002400260025002040F66A17B94242
:1035000000D100BF1846C1F3421401F01F06012785
:1035100007FA06F5012C01D10C3004E0022C01D190
:10352000103000E014301AB107682F43076002E042
:103530000768AF430760F0BD2DE9F04786B0054648
:103540000E460024A24600BFA1460027B08900B164
:1035500000BF2F462C8A4CF6FF700440F0880443CD
:103560002C82AC894EF6F3100440B08831890843B0
:10357000718908430443AC81AC8A4FF6FF40044094
:10358000B0890443AC8201A8FDF728FF1F48874299
:1035900002D1DDF810A001E0DDF80CA0A88900F44C
:1035A000004040B10AEBCA0000EB0A103168490044
:1035B000B0FBF1F807E00AEBCA0000EB0A10316833
:1035C0008900B0FBF1F86420B8FBF0F00401200999
:1035D000642101FB1089A88900F4004040B1322029
:1035E00000EBC900B0FBF1F000F00700044308E075
:1035F000322000EB09106421B0FBF1F000F00F0065
:1036000004432C8106B0BDE8F0870000003801407B
:1036100001468888C0F308007047C1F30802828021
:10362000704700BFFEE7000010B50446240300F019
:10363000B3F800F0A7F800200B4908602020FEF73F
:10364000B5FDC4F30740FEF7B1FDC4F30720FEF754
:10365000ADFDE0B2FEF7AAFD01200449C1F89001DA
:1036600000F090F810BD00009001214200002142BE
:1036700008B501210420FDF78BFE1020ADF80000F5
:103680008DF8030003208DF8020069460948FDF714
:1036900036FB10210748FDF7BFFB012006490860F3
:1036A000FEF73CFD0020FEF7ABFD00F031F80349CA
:1036B000088008BD0008014090012142140000204C
:1036C0002DE9F04106460C46174600200F490860D8
:1036D0000320FEF76BFDC4F30740FEF767FDC4F35C
:1036E0000720FEF763FDE0B2FEF760FD002505E070
:1036F000FF20FEF75BFD7055681C85B2BD42F7DB0D
:10370000012002490860BDE8F081000090012142DB
:1037100010B5002400200E4908609020FEF746FDF9
:103720000020FEF743FD0020FEF740FD0020FEF7DD
:103730003DFDFF20FEF73AFD44EA0024FF20FEF79E
:1037400035FD044301200349C1F89001204610BD16
:10375000900121420000214210B5002400200749B9
:1037600008600520FEF722FDFF20FEF71FFD04463E
:1037700001200349C1F89001204610BD900121426B
:103780000000214210B500BFFFF7E6FF00F0010086
:103790000028F9D110BD000010B5002004490860D0
:1037A0000620FEF703FD01200249C1F8900110BD7B
:1037B00090012142000021422DE9F04107460E46CA
:1037C0001446F0B2C0F58075AC4200DC254612E02C
:1037D0002A463146384600F013F8AC4200D10BE0DF
:1037E0002F442E44601B84B2B4F5807F02DD4FF479
:1037F000807500E02546EBE700BFBDE8F0810000E2
:103800002DE9F04106460C461746FFF7C5FF00209C
:103810000F4908600220FEF7C9FCC4F30740FEF719
:10382000C5FCC4F30720FEF7C1FCE0B2FEF7BEFC06
:10383000002504E0705DFEF7B9FC681C85B2BD424E
:10384000F8DB012002490860FFF79CFFBDE8F0812A
:103850009001214210B5FFF70BFF0020FFF7E4FEB7
:103860006C2200210148FFF7A7FF10BD1A000020BD
:103870000FB4054B10B503A9044A029800F0DAF81A
:1038800010BC5DF814FB0000F5410008EC010020BD
:1038900002E008C8121F08C1002AFAD17047704719
:1038A000002001E001C1121F002AFBD17047000077
:1038B0002DE9FF5F82B00021DDE90430020DDDF863
:1038C00040B0034318D044F61050A2F2FF324243F6
:1038D0001514119801281FD0A5EB0B00401C5FEABE
:1038E000000A4FF000064E4FDFF83891B0465046C0
:1038F00015D5CAF1000413E0119801244AA3012848
:1039000001D16FEA0B010298119AC0E90031C0E9B8
:10391000024206B0BDE8F09FCBF10000DFE70446AD
:103920000021404A491842EB0450CDE9001012E052
:10393000E00707D032463B4640464946FCF7C1FD0A
:103940008046894632463B4610461946FCF7B9FD8B
:1039500006460F466410002CEAD1DDE90401DDE9DA
:103960000023BAF1000F06DAFCF7ABFD42464B46E6
:10397000FCF7A7FD05E0FCF716FE42464B46FCF7B8
:1039800012FE04460E460022284BFCF7E3FE03D845
:103990004FF0FF30014607E00022254B204631461C
:1039A000FCF7E8FCFDF72AF8102409E0002C0ADBFC
:1039B0000A220023FCF72CFF039B30321A55641EA9
:1039C00050EA0102F2D1641C039AC4F111031444B9
:1039D000119A012A03D0012208430DD10AE00843BD
:1039E00004D000204FF0110B119072E7A3EB0B05F0
:1039F0006D1E0DE05B4504DD4FF0000205F1010591
:103A000004E003DA4FF00002A5F10105002AECD032
:103A100002981199C0E90231C0E9004579E7000038
:103A2000000014400000F03F300000000000F043B0
:103A30000000E03F2DE9FF4F95B09A4688460646C4
:103A40000025EEE1252877D100242746F94A0121F7
:103A5000039400E0044316F8013F203B01FA03F011
:103A60001042F7D130782A2811D06FF02F03307828
:103A7000A0F13002092A16D8039A44F0020402EB9E
:103A8000820203EB42021044761C0390EFE758F8E1
:103A9000042B0392002A03DA504244F400540390AA
:103AA00044F00204761C30782E2816D116F8010F47
:103AB00044F004042A280DD06FF02F023078A0F1D2
:103AC0003003092B09D807EB870302EB4303C71820
:103AD000761CF3E758F8047B761C30786C280FD0FE
:103AE00006DC4C2817D068280DD06A2814D104E0D1
:103AF000742810D07A280FD10DE044F400140AE0A5
:103B000044F4801401E044F440147278824202D1FB
:103B100004F58014761C761C307866280BD013DCF4
:103B2000582877D009DC002875D04528F6D04628DB
:103B3000F4D047281AD193E118E0632835D06428DF
:103B400079D0652812D18BE1702873D008DC672802
:103B5000F1D069286FD06E280DD06F2806D1ACE067
:103B600073282CD0752874D0782853D052461799D2
:103B700090476D1C54E1C4F30250022809D0032879
:103B80000DD0D8F8001004280DD00D6008F10408FD
:103B900046E1D8F80010EA17C1E90052F6E7D8F874
:103BA00000100D80F2E70D70F0E718F8041B8DF897
:103BB000001000208DF80100EB46012003E058F8CA
:103BC00004BB4FF0FF3061074FF0000102D40DE05D
:103BD00009F101018946B9420FDA8145F8DB1BF88A
:103BE00009100029F4D108E009F101018946814258
:103BF000FADB1BF809100029F6D103985346A0EB15
:103C0000090721463846179A00F080FA284400EB4D
:103C1000090507E044E008E10DE01BF8010B5246FE
:103C200017999047B9F10109F7D253462146384612
:103C3000179AF2E039E00A21C4F302524FF0000B68
:103C40000091022A06D058F8040BC117032A09D0A4
:103C50000AE023E008F1070020F00702F2E8020181
:103C6000904605E000B2C117042A01D140B2C11745
:103C7000002906DA0A460021404261EB02012D22AA
:103C800002E0220504D52B228DF80420012203E056
:103C9000E20701D02022F7E7914657E00A2100E031
:103CA00010214FF0000B00910BE010214FF0000BA2
:103CB00044F004040827009103E008204FF0000BB3
:103CC0000090C4F30252022A05D058F8040B0021D8
:103CD000032A08D008E008F1070020F00702F2E804
:103CE0000201904603E080B2042A00D1C0B24FF036
:103CF000000922072AD53278702A07D0DDF800C0E3
:103D00008CF0100C5CEA0B0C05D00EE040228DF814
:103D10000420012208E050EA010306D030238DF888
:103D200004308DF8052002229146009B83F00803A1
:103D300053EA0B030AD150EA010201D1620705D50B
:103D400030228DF804204FF001097F1E3278582A66
:103D500004D039A20C920CAA02920BE03BA2F9E724
:103D60005B46009AFCF754FD0C9B9B5C029A521E2A
:103D70000292137050EA0102F2D1029804A9081AC3
:103D800000F1200B600702D524F4803400E0012705
:103D90005F4502DDA7EB0B0000E0002000EB0B010C
:103DA000009003984944401A0390E00306D4534618
:103DB0002146179A039800F0A9F90544002706E068
:103DC00001A85246C05D179990476D1C7F1C4F4556
:103DD000F6DBE0030CD553462146179A039800F012
:103DE00095F9054404E030205246179990476D1C20
:103DF0000099481E00900029F5DC08E0029802991D
:103E000052460078491C0291179990476D1CBBF1EE
:103E10000001ABF1010BF1DC5BE100F065F9054459
:103E2000761C307800287FF40DAE19B02846BDE826
:103E3000F08F000009280100303132333435363735
:103E400038396162636465660000000030313233E6
:103E50003435363738394142434445460000000086
:103E6000600700D4062708F1070020F00700F0E8FB
:103E70000223804603F0004C5FEA0C0001D097A0BB
:103E800009E0200501D596A005E0E00701D095A046
:103E900001E0AFF24C001390307823F00043652826
:103EA0000CD006DC452809D046281DD047287FD1F4
:103EB0003BE0662818D067287AD136E00021112F20
:103EC00001DB112000E0781CCDE9000104A90CA859
:103ED000FFF7EEFCDDE90D010C9A4FF0000B07F146
:103EE0000109109200914EE04FF000400097CDE99B
:103EF000011004A90CA8FFF7DBFCDDE90D020C9B07
:103F00000F994FF0000B91461093009211B9791C54
:103F100000EB0109B7EB090003D4C0F1FF3B07F147
:103F20000109A9EB0700019042E0012F00DA012707
:103F30000021112F01DD112000E03846CDE90001FC
:103F400004A90CA8FFF7B4FCDDE90D010C9A00915F
:103F50004FF0000BB946109221070FD4009A4A4542
:103F600003DA914601E0A9F10109B9F1010F05DD7C
:103F7000109AA9F10101515C3029F4D0B84202DA5B
:103F800010F1040F03DA0121CDE9011010E000283F
:103F900003DC8344A9EB000102E0411C494500DD3C
:103FA0008946A0EB0B00401C01904FF000400290AE
:103FB000200705D40198484502DB4FF0FF300190FF
:103FC00000208DF84B0002980DF14B07B0F1004F27
:103FD00025D002200C902B200D90029800280CDA9E
:103FE000404202902D200D9007E00A210298FCF734
:103FF000F9FB3031029007F8011D0C99481E0C9016
:104000000029F2DC02980028EFD1791E0D98087083
:10401000307800F0200040F0450007F8020D11A8AC
:10402000C01BC01D02901398007800B1012000EB66
:104030000901019801EBE071029801440398401ACC
:10404000401E0390E00306D453462146179A039876
:1040500000F05CF805441398007818B1524617999F
:1040600090476D1CE00323D553462146179A0398C9
:1040700000F04CF805441BE0BBF1000F07DB009893
:10408000584504DD1098179910F80B0001E01799B6
:1040900030205246904701980BF1010B401E05F16C
:1040A0000105019004D12E205246179990476D1CAE
:1040B000B9F10001A9F10109DEDC05E017F8010BF7
:1040C0005246179990476D1C0299481E029000298C
:1040D000F4DC53462146179A03989EE62D00000013
:1040E0002B000000200000002DE9F04104460025CF
:1040F0001E461746880404D405E039462020B04700
:104100006D1C641EF9D52846BDE8F0812DE9F0410B
:10411000044600251E469046C80301D5302700E01E
:104120002027880404D505E041463846B0476D1C79
:10413000641EF9D52846BDE8F08170B50446002517
:10414000104603E00E5C66556D1C401C9842F9DB7E
:1041500070BD000070B5044602F032F8012810D09E
:104160000B480088844206D309480088B4FBF0F568
:10417000284601F0A9F906480088B4FBF0F100FBDD
:1041800011444FF47A7104FB01F000F003F870BDA4
:10419000D600002070B5034600224FF0E026756976
:1041A0000D4E367803FB06F44FF0E026B16910E0BF
:1041B0004FF0E026B06988420BD0884202D20E1A36
:1041C000324402E02E1A0E4432440146A24200D389
:1041D00000E0EDE700BF70BDD400002030B504461C
:1041E000002504E04FF47A70FFF7D4FF6D1CA54260
:1041F000F8D330BD70B504460D460120084908606B
:10420000E1B20848FFF709FA00BF80210548FFF72F
:1042100037F90028F9D0002001490860204670BD18
:10422000A4812142004400401FB54FF44070FCF7C8
:10423000BFFE4820FEF7C8FC4FF41660FFF7B0F849
:10424000FCF778FF32A0FFF713FB40F2671140F252
:104250008F10FEF7FDFF4FF49650FDF795F9FCF730
:10426000DDFDFDF761FDFEF721FD44F62060FFF75F
:1042700071FFFDF71BFF28482849294A294BCDE942
:104280000032CDE90210284B284A29492948FCF779
:1042900047FCFFF7DFFA40F2CF2140F2F310FCF7C2
:1042A0005BFF40F2CF2140F2F310FCF7A7FF40F292
:1042B000CF2140F2F310FCF7F3FF41F61F4142F229
:1042C0000F70FEF7A5FD0220FCF7D0FDC8211A48AB
:1042D000FEF769FF42F21070FFF780FF0020FDF744
:1042E00025F80020FDF72CF80020FDF731F84FF4F9
:1042F000FA70FFF72FFF1E20FDF718F81E20FDF7BC
:104300001FF81E20FDF724F800F018F800BFFEE7A4
:10431000B8B4CEBB0D0A0000840100208201002049
:10432000800100207E0100207C0100208701002008
:10433000860100207A010020000800401CB508A07A
:10434000FFF796FA0B4800210B468022CDE90010BA
:1043500009A10C4801F004FF01F052FA1CBD000055
:10436000C8EBBFDABAAFCAFDB5F7D3C3B3C9B9A6B4
:104370000D0A0000B401002073746172745F7461EF
:10438000736B0000095000082DE9F04105460E4608
:104390001C4807681C480068001D00F0D7FE50B993
:1043A0001948006890F82C100120884017490968C6
:1043B000814316480160681C38B936B1124801685B
:1043C000091D134800F000FF1AE07C190E48006830
:1043D0004460BC4207D20C480168091D0D480068C2
:1043E00000F0D8FE0CE008480168091D0A48006882
:1043F00000F0D0FE09480068844201D207480460FA
:10440000BDE8F08104010020F00000200801002038
:104410007C070020F8000020F4000020200100208C
:1044200010B5044600F0DCFE23480068401C224919
:1044300008602248006840B92048046008460068C7
:1044400001280DD100F0E4F90AE01D48006838B9F0
:104450001A480068C06AE16A884201D817480460B7
:1044600018480068401C1749086094F82C10012077
:10447000884015490968084313490860E16A01EB5F
:104480008101124A02EB8100211D00F09DFE00F027
:10449000EBFE0B48006868B108480068C06AE16A32
:1044A000884207D24FF0805009490860BFF34F8F10
:1044B000BFF36F8F10BD000000010020F00000204E
:1044C0000C0100201C01002008010020AC04002089
:1044D00004ED00E010B500F083FE10480068D0B98C
:1044E0000F4800F047FE0F4800F044FE0C480E490C
:1044F00008600C480D49086000220C210A2001F0D8
:104500009BFA064908600846006820B108A10348E4
:10451000006800F09DFF00F0A7FE10BD34010020F0
:1045200090070020A40700202C010020300100206B
:10453000546D72510000000070B523E001F0B6F92F
:104540001348006808B9012000E00020054601F08A
:10455000C3FFBDB900F044FE0D48C068C468201D0B
:1045600000F0F4FD0B480068401E0A4908600A4844
:104570000068401E0849086000F076FE204600F002
:1045800060F800BF044800680028D7D170BD000063
:104590006807002000010020FC00002070B50446E0
:1045A0000D46206C70B1216CE0680844E0606168E1
:1045B000E068884201D32068E0602846226CE16808
:1045C000FBF7FEFD70BD2DE9F04104460F46154690
:1045D0004FF00008A66B206C40B9206860BB606893
:1045E00001F0B4FE80460020606025E07DB93946C8
:1045F000226CA068FBF7E4FD216CA0680844A06071
:10460000D4E90110884217D32068A06014E039462D
:10461000226CE068FBF7D4FD216CE068401AE06092
:104620002168E068884203D2216C6068401AE0602B
:10463000022D01D106B1761E701CA0634046BDE874
:10464000F08110B50446206B00F046FE204600F0D5
:1046500043FE10BD0146084A126812680AB90122D9
:1046600000E000220A600A6822B9034A1268D26890
:10467000106800E0002070472C01002030B54FF496
:104680002053174800F007042CB1C01D20F007008C
:10469000134C041B1B1B0246124C22600024114DBC
:1046A0006C60D018083820F007000F4C2060002400
:1046B0000D4D2D686C600C4D2D682C601146441A10
:1046C0004C60094C24680C60084D4C682C60084D07
:1046D0004C682C604FF00044064D2C6030BD00004B
:1046E000080800204C010020540100205C0100203B
:1046F000580100206001002000BFFFF71DFF0648A1
:1047000000680128F9D94FF0805004490860BFF3D0
:104710004F8FBFF36F8FF0E7AC04002004ED00E093
:104720002DE9F04106460D4617469846069C0DB900
:10473000246000E02760E66325640121204601F043
:10474000C1FA0020A064BDE8F08100002DE9FF5F00
:1047500081460F469246DDE90E6B109CAAF10100DE
:10476000216B01EB800828F0070808F0070008B962
:10477000012000E0002028B940F22B321BA120A02C
:10478000FFF776F8002507E0795D04F13400415524
:10479000785D00B902E06D1C102DF5D300BF00213B
:1047A00043200155202E00D31F26E66266640020B8
:1047B000A064201D00F0EBFC04F1180000F0E7FC01
:1047C0002461C6F12000A06164620020E06484F8E6
:1047D000500049464046039A00F004FC2060BBF1BB
:1047E000000F01D0CBF80040BDE8FF9F2E2E5C46A5
:1047F00072656552544F535C7461736B732E630022
:104800004572726F723A25732C25640D0A00000000
:1048100010B5002407E004EB84010F4A02EB81008D
:1048200000F0A8FC641C202CF5D30C4800F0A2FC7E
:104830000B4800F09FFC0B4800F09CFC0A4800F07D
:1048400099FC0A4800F096FC0448094908600448AD
:104850000849086010BD0000AC0400202C070020AF
:104860004007002054070020680700207C07002034
:10487000F4000020F800002010B50146164800E0C2
:10488000006803688B42FBD30246436813448B42A3
:1048900004D143684C682344436001460A464B6890
:1048A00013440468A34211D10C4C03682468A3424A
:1048B00008D04B680468646823444B6003681B6835
:1048C0000B6005E0054B1B680B6001E003680B60A3
:1048D000884200D0016010BD4C010020540100202E
:1048E0002DE9F04104460D4616461F464FF00008DC
:1048F00065602461B5420CD8F01BA169884202D3DF
:104900004FF0010811E0211D0948006800F042FC49
:104910000BE0BE4204D2BD4202D34FF0010804E0D6
:10492000211D0448006800F035FC4046BDE8F081D8
:10493000300100202C01002070B5054600F050FC2D
:10494000A86B08B9012400E0002400F08DFC20468B
:1049500070BD70B5054600F043FCA86BE96B88425A
:1049600001D1012400E0002400F07EFC204670BD4F
:104970002DE9F3410D460098846C00272CB940F6D0
:10498000CE121AA128A0FEF773FFA06BE16B88423C
:1049900001D2012000E0002028B940F6CF1213A177
:1049A00021A0FEF765FFA06BE16B88421BD294F952
:1049B00045602A4669462046FFF705FE0746701CFB
:1049C00060B9606A08B9012000E0002050B904F124
:1049D000240001F027FD28B1012703E0701C40B23C
:1049E00084F8450000BF3846BDE8FC812E2E5C2EC1
:1049F0002E5C2E2E5C73746D33322D636F6E747269
:104A00006F6C205F6C69616E77616E675C636F6E5F
:104A100074726F6C5C4672656552544F535C71756D
:104A20006575652E630000004572726F723A2573DA
:104A30002C25640D0A000000F8B505460F46134802
:104A40000068C068C468201D00F080FBE069012890
:104A500018D1A06941192B463A462046FFF740FF7E
:104A600080B1002003462A4601460090204601F00E
:104A7000FDFD06462EB94FF4027205A10AA0FEF70D
:104A8000F7FE00BF2046616A8847F8BD2C01002070
:104A90002E2E5C4672656552544F535C74696D6589
:104AA00072732E63000000004572726F723A2573B4
:104AB0002C25640D0A00000070B586B060E00398F4
:104AC00000285DDB059C606908B9012000E000203A
:104AD00010B9201D00F03AFB02A800F0C7F8054607
:104AE00003980A284AD2DFE800F00905072C2E4572
:104AF00006082D2F00BF00BF00BF00BF0498A269A9
:104B0000811803462A462046FFF7EAFEC0B1204638
:104B1000616A8847E069012812D10020009004985A
:104B2000A169421800231946204601F09FFD064660
:104B30002EB940F2213218A11DA0FEF799FE00BF48
:104B40001DE000BF1BE000BF0498A061A06908B190
:104B5000012000E0002028B94FF44E720EA114A0ED
:104B6000FEF786FEA06941192B462A462046FFF72C
:104B7000B7FE04E0204600F0AFFB00E000BF00BF3E
:104B800000231A4603A90E48006800F0A3FF00287E
:104B900095D106B070BD00002E2E5C467265655240
:104BA000544F535C74696D6572732E63000000008E
:104BB0004572726F723A25732C25640D0A0000004D
:104BC00034010020F8B505460C4600F06FFE68463B
:104BD00000F04CF80646009820BB44B9B54206D810
:104BE00001F07AFC31462846FFF726FF1CE03CB175
:104BF0000E480068006808B9012000E00020044663
:104C0000A91B22460A48006800F038FC01F064FC49
:104C100050B94FF0805007490860BFF34F8FBFF382
:104C20006F8F01E001F058FCF8BD0000300100205A
:104C30003401002004ED00E00A490968096809B957
:104C4000012100E0002121B14FF0FF31064A11603F
:104C500006E004490968C968C868034A41681160E8
:104C600070470000F40000202001002070B50446C9
:104C700001F0B6FA054607480068854204D200F004
:104C80000BF80120206001E0002020600148056051
:104C9000284670BD3C0100202DE9F8432DE0214855
:104CA0000068C06805681F480068C068C468201DA7
:104CB00000F04CFA2046616A8847E06901281CD15F
:104CC000A0694619AE4207D966602461211D1548C6
:104CD000006800F05FFA10E0002003462A46014613
:104CE0000090204601F0C2FC07462FB940F29232F4
:104CF0000DA113A0FEF7BCFD00BF0A4800680068C4
:104D000008B9012000E000200028C8D00548D0F8EC
:104D100000800F480068034908600D48C0F8008013
:104D2000BDE8F8832C0100202E2E5C46726565528A
:104D3000544F535C74696D6572732E6300000000FC
:104D40004572726F723A25732C25640D0A000000BB
:104D5000300100200B480068401C08B9012000E029
:104D6000002020B9F42208A112A0FEF781FD00BFA7
:104D7000502080F31188BFF34F8FBFF36F8F00BFB8
:104D800000BFFEE7400100202E2E5C467265655292
:104D9000544F535C706F727461626C655C52564420
:104DA000535C41524D5F434D335C706F72742E63A0
:104DB000000000004572726F723A25732C25640D55
:104DC0000A00000008B500BF6846FFF743FC044630
:104DD00020460099FFF7F6FEFFF76EFEF4E770B588
:104DE000044600F0FDF994F945501AE0A06C38B182
:104DF00000212046FFF7BCFD88B100F025FC0EE045
:104E0000606A08B9012000E0002038B904F12400EC
:104E100001F008FB18B100F017FC00E003E0681E89
:104E200045B2002DE2DC00BFFF2084F8450000F011
:104E30001BFA00F0D5F994F9445010E0206908B944
:104E4000012000E0002048B904F1100001F0EAFA66
:104E500008B100F0F9FB681E45B200E001E0002D4A
:104E6000ECDC00BFFF2084F8440000F0FDF970BDC9
:104E70002DE9F04104464FF0000800F017FD3E48D0
:104E8000006808B9FFF7FAFB3C480068204000289A
:104E90005FD1A4B1083404F0070080B104F007002A
:104EA000C0F10800044404F0070008B9012000E044
:104EB000002020B9BF2232A13BA0FEF7D9FC002C74
:104EC00047D03D480068844243D83C4E3046056890
:104ED00001E02E462D686868A04202D228680028AA
:104EE000F7D125480068854233D0306800F10808C2
:104EF000286830606868001B102813D92F1907F044
:104F0000070008B9012000E0002020B9EC221CA114
:104F100025A0FEF7ADFC6868001B78606C60384621
:104F2000FFF7AAFC244968680968081A2249086042
:104F30000846006822490968884203D21E48006872
:104F40001F4908600D4968680968084368600020C7
:104F5000286001F0C1FA08F0070008B9012000E05C
:104F6000002028B94FF4967205A10FA0FEF780FC2F
:104F70004046BDE8F081000054010020600100209F
:104F80002E2E5C4672656552544F535C706F72747E
:104F900061626C655C4D656D4D616E675C686561F5
:104FA000705F342E630000004572726F723A257391
:104FB0002C25640D0A000000580100204C0100203F
:104FC0005C0100200648006830B10549096801F11C
:104FD0004800896C491C0160014800687047000066
:104FE000F0000020001F4FF080730360001F21F0CD
:104FF00001030360001F034B036014380260203874
:1050000070470000554D00081CB5044600F0E8F854
:105010000E48012100234A02CDE900100CA11348DB
:1050200001F09EF81249086008460068012803D183
:1050300010A0FEF71DFC02E015A0FEF719FC1B48AE
:10504000006800F07BFA00F00FF91CBDB8010020E9
:1050500053656E736F725F436F6D6D756E696361DB
:1050600074696F6E5F7461736B0000009D220008AD
:10507000BC010020D3EBB4ABB8D0C6F7CDA8D0C5E7
:10508000C8CECEF1B4B4BDA8B3C9B9A60D0A00000C
:10509000D3EBB4ABB8D0C6F7CDA8D0C5C8CECEF14F
:1050A000B4B4BDA8CAA7B0DC0D0A0000B40100204A
:1050B0001CB520492048FCF7E3FC1F480078C0EBF2
:1050C00000101C49097801EB80001C4908801C482D
:1050D000007800EBC00040000E381A49095C1848FF
:1050E000007800EBC00040000F38164A105CC0EB9F
:1050F000001001EB800014490880104800880988DE
:10510000884214DB0020009003460122092101900F
:1051100040F2E770FCF72EFF09480078062801D11D
:1051200001201CBD06480078401CC0B2F9E70448C5
:105130000078F6E7730100207201002016000020BD
:105140007A0100201A0000201800002001460A6998
:10515000D1E901309860D1E9010358605068884274
:1051600001D188685060002008611068401E1060FE
:105170001068704700F1080141604FF0FF31816015
:1051800000F10801C1600161002101607047002148
:105190000161704710B502460B685C1C0CB91069C0
:1051A00007E002F1080000E04068446824689C427F
:1051B000FAD944684C604C68A160886041600A611B
:1051C0001468641C146010BD42684A6093688B6068
:1051D000936859609160086103685B1C03607047C5
:1051E00010B500BF502080F31188BFF34F8FBFF37D
:1051F0006F8F00BF0B480068401C0A4908600846D2
:10520000006801280DD108480068C0B208B9012023
:1052100000E0002028B94FF4BD7204A10EA0FEF7F3
:1052200027FB10BD4001002004ED00E02E2E5C465F
:1052300072656552544F535C706F727461626C6535
:105240005C525644535C41524D5F434D335C706F2A
:1052500072742E63000000004572726F723A2573FB
:105260002C25640D0A00000010B50B48006828B911
:1052700040F2811209A114A0FEF7FAFA064800686C
:10528000401E054908600846006820B9002080F3E8
:10529000118800BF00BF10BD400100202E2E5C46CB
:1052A00072656552544F535C706F727461626C65C5
:1052B0005C525644535C41524D5F434D335C706FBA
:1052C00072742E63000000004572726F723A25738B
:1052D0002C25640D0A00000070B506463546002EE8
:1052E00035D0083D2C461A4960680968084008B165
:1052F000012000E0002028B94FF4A07215A11FA0E2
:10530000FEF7B6FA206808B9012000E0002028B9AD
:1053100040F241120FA119A0FEF7AAFA0C496068E9
:105320000968084098B1206888B909496068096827
:105330008843606000F0BAFA14496068096808445C
:10534000124908602046FFF797FA01F0C5F870BDD2
:10535000600100202E2E5C4672656552544F535CEE
:10536000706F727461626C655C4D656D4D616E67E6
:105370005C686561705F342E630000004572726F77
:10538000723A25732C25640D0A0000005801002094
:10539000064800684FF47A71B0FBF1F0401E4FF000
:1053A000E0214861072008617047000000000020EC
:1053B00070B5FAF7EFFE0546102D11D305F1E02088
:1053C00090F8F04310480078844201DB012000E0AF
:1053D000002028B94FF42A720CA117A0FEF748FA52
:1053E0001948006800F4E06018490968884201D84B
:1053F000012000E0002028B94FF42E7203A10EA076
:10540000FEF736FA70BD0000440100202E2E5C46E7
:1054100072656552544F535C706F727461626C6553
:105420005C525644535C41524D5F434D335C706F48
:1054300072742E63000000004572726F723A257319
:105440002C25640D0A0000000CED00E0480100204E
:10545000024600200BE0084B53F8303033B9064BBE
:1054600043F8301003EBC0035A6002E0401C0A28E6
:10547000F1D300BF70470000B80700202DE9F041CC
:1054800005460E4617462C46FFF7AAFE94F944003F
:10549000401C10B9002084F8440094F94500401CD9
:1054A00010B9002084F84500FFF7DEFEA06B28B994
:1054B0003A46314604F1240000F0F6F82046FFF7A2
:1054C0008EFCBDE8F081000070B504460025ACB14B
:1054D0000F48006808B9012000E0002028B940F218
:1054E000CF420CA110A0FEF7C3F900F0DFF90021B4
:1054F0002046FEF749FF00F0EFFF05463DB94FF0AB
:1055000080500D490860BFF34F8FBFF36F8F70BDA0
:10551000280100202E2E5C4672656552544F535C64
:105520007461736B732E63004572726F723A2573E8
:105530002C25640D0A00000004ED00E070B505465E
:10554000FFF74EFE15B92D48006800E028460446D6
:10555000201DFFF7FBFD78B9E06A00EB80002849C9
:1055600051F8200040B994F82C10012088402549BA
:105570000968814323480160A06A18B104F118004A
:10558000FFF7E4FD20480068401C1F4908601B48E5
:105590000068844209D1211D1C48FFF715FE1C48F4
:1055A0000068401C1A49086009E01A480068401E5B
:1055B000184908602046FFF744F8FFF73DFBFFF766
:1055C00053FE15480068C0B10C480068844214D1ED
:1055D0001248006808B9012000E0002028B940F214
:1055E00065420FA113A0FEF743F94FF08050154913
:1055F0000860BFF34F8FBFF36F8F70BDF0000020C6
:10560000AC040020080100201C01002068070020D5
:10561000FC000020000100200C01002028010020D7
:105620002E2E5C4672656552544F535C7461736BE9
:10563000732E63004572726F723A25732C25640DC8
:105640000A00000004ED00E00120014908607047F5
:105650001401002070B504460D462CB940F6063200
:1056600007A10CA0FEF704F90E4801681831204686
:10567000FFF790FD01212846FEF786FE70BD000071
:105680002E2E5C4672656552544F535C7461736B89
:10569000732E63004572726F723A25732C25640D68
:1056A0000A000000F000002070B505460E461446C2
:1056B0002DB940F6313209A10DA0FEF7D9F81048F6
:1056C000016818312846FFF77FFD0CB14FF0FF3617
:1056D00021463046FEF758FE70BD00002E2E5C4677
:1056E00072656552544F535C7461736B732E630023
:1056F0004572726F723A25732C25640D0A00000002
:10570000F000002070B505462C46002D4BD02649F0
:10571000E06A0968C96A884245D2A06900F0004081
:1057200028B921480068C06AC0F12000A061E16A80
:1057300001EB81011D4A02EB81016069884201D1C0
:10574000012000E0002050B3201DFFF7FFFC78B9D6
:10575000E06A00EB8000154951F8200040B994F848
:105760002C100120884012490968814310480160CB
:105770000D480068C06AE06294F82C10012088404F
:105780000B49096808430A490860E16A01EB810195
:10579000064A02EB8100211DFFF716FD03E00248D7
:1057A0000068C06AE06270BDF0000020AC04002018
:1057B0000801002010B504462CB940F6C13205A1FD
:1057C00009A0FEF755F80C48006820600B480068F7
:1057D000606010BD2E2E5C4672656552544F535C5E
:1057E0007461736B732E63004572726F723A257326
:1057F0002C25640D0A00000018010020040100207F
:105800001CB51A4800210B468022CDE9001018A1D2
:10581000194800F0A5FC0446012C02D100F0ECFE72
:105820000446012C15D100BF502080F31188BFF32E
:105830004F8FBFF36F8F00BF4FF0FF300F490860ED
:1058400001200F49086000200E49086000F08AF826
:105850000BE0601C08B1012000E0002028B940F2F4
:10586000847209A10DA0FEF703F81CBD24010020DD
:1058700049444C4500000000F94600082001002082
:105880000C010020040100202E2E5C46726565523A
:10589000544F535C7461736B732E63004572726F67
:1058A000723A25732C25640D0A0000000248006836
:1058B000401C0149086070472801002010B51B48B2
:1058C000006818B101201A4908602DE0002018492D
:1058D000086018480068B0FA80F0C0F11F0404EBBB
:1058E0008400154951F8200008B1012000E0002093
:1058F00028B940F6F62211A115A0FDF7B9FF04EB77
:1059000084010D4A02EB810041684968416000F161
:10591000080142688A4202D1416849684160416891
:10592000C9680F4A116000BF10BD000028010020A7
:105930001401002008010020AC0400202E2E5C463B
:1059400072656552544F535C7461736B732E6300C0
:105950004572726F723A25732C25640D0A0000009F
:10596000F00000201CB52248014609780191FF2172
:10597000024611700146097800919DF8001001F06F
:1059800050011C4A117007211B4A116009E01A4995
:105990000968491E184A11609DF800104906090E51
:1059A00000919DF8001001F080018029EFD012498C
:1059B00009680902104A11601146098801F4E06182
:1059C00011600B4A019911700C48006840F4700096
:1059D0000A4908600846006840F070400860FFF718
:1059E000D7FC002006490860FAF79EFB00201CBD8A
:1059F00000E400E0440100204801002020ED00E028
:105A00004001002010B500BF502080F31188BFF383
:105A10004F8FBFF36F8F00BF00F0E8FB18B14FF05E
:105A200080500449086000BF002080F3118800BF47
:105A300010BD000004ED00E02DE9F84305460E46D8
:105A400090460DB1012000E0002028B94FF4C47247
:105A50000DA11CA0FDF70CFF0EB9002701E005FB0E
:105A600006F707F14C00FFF703FA044644B104F1CE
:105A70004C0943464A46314628460094FEF750FEFC
:105A80002046BDE8F88300002E2E5C2E2E5C2E2EC4
:105A90005C73746D33322D636F6E74726F6C205F44
:105AA0006C69616E77616E675C636F6E74726F6C48
:105AB0005C4672656552544F535C71756575652E11
:105AC000630000004572726F723A25732C25640DD5
:105AD0000A0000002DE9FF4782B005460E461F462A
:105AE0004FF0000A2C462CB940F2DC4261A170A0B4
:105AF000FDF7BEFE0EB9206C08B9012000E00020C1
:105B000028B940F2DD425BA169A0FDF7B1FE00F0CB
:105B100057FB08B9049808B9012000E0002028B913
:105B20004FF49C6253A162A0FDF7A2FE00BFFFF7F5
:105B300057FBD4F83890B9F1000F3DD0D4F80C8061
:105B400031462046FEF72AFDDFB9A9F10100A06326
:105B5000206810B9FFF736FA6060206908B90120A3
:105B600000E0002010BB04F1100000F05BFCE8B185
:105B70004FF0805052490860BFF34F8FBFF36F8FD3
:105B800014E0C4F80C80606A08B9012000E000202D
:105B900060B904F1240000F045FC38B14FF08050AA
:105BA00047490860BFF34F8FBFF36F8FFFF75CFB70
:105BB000012006B0BDE8F087049818B9FFF754FB40
:105BC0000020F6E7BAF1000F04D16846FFF7F2FDB6
:105BD0004FF0010AFFF748FBFFF768FEFFF700FBF5
:105BE00094F94400401C10B9002084F8440094F952
:105BF0004500401C10B9002084F84500FFF734FB35
:105C000004A9684600F05CFA40BB2046FEF794FE0B
:105C1000F0B1206830B9FFF7E3FA6068FFF772FD72
:105C2000FFF722FB04F124000499FFF713FD20463F
:105C3000FFF7D5F800F050FC00287FF478AF4FF064
:105C400080501F490860BFF34F8FBFF36F8F6EE71F
:105C50002046FFF7C4F800F03FFC68E72046FFF756
:105C6000BEF800F039FC2046FEF766FE0028EED0B4
:105C700000209EE72E2E5C2E2E5C2E2E5C73746D03
:105C800033322D636F6E74726F6C205F6C69616E5E
:105C900077616E675C636F6E74726F6C5C46726581
:105CA0006552544F535C71756575652E6300000035
:105CB0004572726F723A25732C25640D0A0000003C
:105CC00004ED00E070B505460E462C462CB940F2B6
:105CD0001B121EA12CA0FDF7CBFDFFF781FAD4E922
:105CE0000F12206801FB020060600020A0632068A2
:105CF000A060E06B401E226C216800FB0210E06097
:105D0000FF2084F8440084F845009EB9206908B952
:105D1000012000E00020A8B904F1100000F082FB8F
:105D200080B14FF080501C490860BFF34F8FBFF324
:105D30006F8F07E004F11000FFF71CFA04F1240054
:105D4000FFF718FAFFF790FA012070BD2E2E5C2E97
:105D50002E5C2E2E5C73746D33322D636F6E7472F5
:105D60006F6C205F6C69616E77616E675C636F6EEC
:105D700074726F6C5C4672656552544F535C7175FA
:105D80006575652E630000004572726F723A257367
:105D90002C25640D0A00000004ED00E02DE9FF430E
:105DA00083B0064688461D464FF0000934462CB99C
:105DB00040F2D92260A16FA0FDF75AFDB8F1000FA3
:105DC00001D1206C08B9012000E0002028B940F280
:105DD000DA2259A167A0FDF74BFD022D02D1E06B3D
:105DE000012801D1012000E0002028B940F2DB2287
:105DF00051A160A0FDF73CFD00F0E2F908B905985B
:105E000008B9012000E0002028B940F2DE224AA1B2
:105E100058A0FDF72DFD00BFFFF7E2F9A06BE16B85
:105E2000884201D3022D38D12A4641462046FEF74A
:105E3000CAFB0746A06C68B129462046FEF798FDCC
:105E400028B34FF080504F490860BFF34F8FBFF326
:105E50006F8F1CE0606A08B9012000E0002068B97B
:105E600004F1240000F0DEFA88B14FF0805045497B
:105E70000860BFF34F8FBFF36F8F08E03FB14FF063
:105E8000805040490860BFF34F8FBFF36F8FFFF71B
:105E9000EBF9012007B0BDE8F083059818B9FFF7CA
:105EA000E3F90020F6E7B9F1000F04D101A8FFF7EC
:105EB00081FC4FF00109FFF7D7F9FFF7F7FCFFF777
:105EC0008FF994F94400401C10B9002084F8440074
:105ED00094F94500401C10B9002084F84500FFF7F4
:105EE000C3F905A901A800F0EBF8F0B92046FEF7C8
:105EF00030FDA0B104F110000599FFF7ABFB20467F
:105F0000FEF76DFF00F0E8FA002885D14FF08050D1
:105F10001C490860BFF34F8FBFF36F8F7CE72046AB
:105F2000FEF75DFF00F0D8FA76E72046FEF757FF50
:105F300000F0D2FA0020ADE72E2E5C2E2E5C2E2E25
:105F40005C73746D33322D636F6E74726F6C205F8F
:105F50006C69616E77616E675C636F6E74726F6C93
:105F60005C4672656552544F535C71756575652E5C
:105F7000630000004572726F723A25732C25640D20
:105F80000A00000004ED00E02DE9F05F80468A463B
:105F900015461E4644462CB940F29F3235A144A016
:105FA000FDF766FCBAF1000F01D1206C08B90120A1
:105FB00000E0002028B94FF468722EA13CA0FDF744
:105FC00057FC022E02D1E06B012801D1012000E034
:105FD000002028B940F2A13226A135A0FDF748FCE7
:105FE000FFF7E6F900BF5021EFF3118081F311882C
:105FF000BFF34F8FBFF36F8F00BF0746A06BE16BFE
:10600000884201D3022E2BD194F945B03246514635
:106010002046FEF7D8FA0BF10100C8B9A06C40B1D8
:1060200031462046FEF7A4FCB8B1B5B10120286086
:1060300013E0606A08B9012000E0002068B904F1AB
:10604000240000F0EFF940B13DB10120286004E0E8
:106050000BF1010040B284F845004FF0010901E066
:106060004FF0000900BF87F3118800BF4846BDE824
:10607000F09F00002E2E5C2E2E5C2E2E5C73746D15
:1060800033322D636F6E74726F6C205F6C69616E5A
:1060900077616E675C636F6E74726F6C5C4672657D
:1060A0006552544F535C71756575652E6300000031
:1060B0004572726F723A25732C25640D0A00000038
:1060C0002DE9F04104460D462CB940F6CB3219A11A
:1060D0001DA0FDF7CDFB2DB940F6CC3215A11AA0BD
:1060E000FDF7C6FBFFF77CF81B4807682868401CD3
:1060F00008B9002619E0194920680968884204D0C7
:106100006068B84201D801260FE06068381A296833
:10611000884209D228686168791A401A28602046A6
:10612000FFF748FB002600E00126FFF79DF8304608
:10613000BDE8F0812E2E5C4672656552544F535C6B
:106140007461736B732E63004572726F723A2573BC
:106150002C25640D0A000000040100201801002015
:106160002DE9FF4F85B0804689461746DDE912AB21
:10617000B800FEF77DFE064656B15420FEF778FEC5
:1061800004460CB1266304E03046FFF7A5F800E0B2
:1061900000247CB10020CDE900ABCDE902403A46B5
:1061A00049464046089BFEF7D1FA2046FEF738F9EB
:1061B000012501E04FF0FF35284609B0BDE8F08F1A
:1061C0000549096809B9012005E00449096809B9C8
:1061D000022000E0002070470C0100202801002070
:1061E0000149086870470000040100202DE9F041D2
:1061F0004FF0000841480068002872D1404800680C
:10620000451C3F480560EDB93E480068006808B984
:10621000012000E0002028B940F6D9123AA13FA0A1
:10622000FDF726FB37480768404800683549086095
:106230003E4807603E480068401C3D490860FEF744
:10624000FBFC00BF3B48006885423CD300BF2D48A3
:106250000068006808B9012000E0002020B14FF07C
:10626000FF30344908602DE026480068C068C468E3
:106270006668B54202D22F48066023E0201DFEF773
:1062800065FFA06A18B104F11800FEF75FFF94F8EB
:106290002C100120884028490968084326490860D5
:1062A000E16A01EB8101254A02EB8100211DFEF725
:1062B0008BFF2349E06A0968C96A8842C7D34FF057
:1062C0000108C4E700BF1E480068C06A00EB8000F8
:1062D0001A4951F82000012801D94FF0010805E0C2
:1062E000FFE718480068401C164908601648006817
:1062F00008B14FF001084046BDE8F08128010020B8
:1063000004010020F40000202E2E5C4672656552C8
:10631000544F535C7461736B732E63004572726FDC
:10632000723A25732C25640D0A000000F800002045
:10633000180100202001002008010020AC040020EA
:10634000F0000020100100201401002070B5054667
:106350002C460026002D4BD026480068844201D1EF
:10636000012000E0002028B940F6C76222A127A042
:10637000FDF77EFAA06C28B940F6C9621EA123A0E1
:10638000FDF776FAA06C401EA064616CE06A88425A
:106390002ED0A06C60BB201DFEF7D8FE78B9E06A55
:1063A00000EB80001D4951F8200040B994F82C10F2
:1063B000012088401A490968814319480160606CCE
:1063C000E062E06AC0F12000A06194F82C10012086
:1063D000884013490968084311490860E16A01EBE4
:1063E00081010E4A02EB8100211DFEF7EDFE012620
:1063F000304670BDF00000202E2E5C46726565525E
:10640000544F535C7461736B732E63004572726FEB
:10641000723A25732C25640D0A000000AC0400209C
:106420000801002070B50646F068C4682CB940F633
:1064300061321AA11EA0FDF71BFA04F11800FEF745
:1064400085FE1F480068A8B9201DFEF77FFE94F85E
:106450002C10012088401B4909680843194908602D
:10646000E16A01EB8101184A02EB8100211DFEF770
:10647000ABFE04E004F118011448FEF7A5FE144930
:10648000E06A0968C96A884204D9012501201149D6
:10649000086000E00025284670BD00002E2E5C46F6
:1064A00072656552544F535C7461736B732E630055
:1064B0004572726F723A25732C25640D0A00000034
:1064C0002801002008010020AC040020540700200F
:1064D000F00000201401002070B50024002634488C
:1064E000006828B94FF4FD6232A137A0FDF7C0F96A
:1064F000FEF776FE2E480068401E2D4908600846CB
:10650000006800284FD13448006800284BD024E0B0
:106510003248C068C46804F11800FEF717FE201D59
:10652000FEF714FE94F82C10012088402C490968CD
:1065300008432B490860E16A01EB8101294A02EB1B
:106540008100211DFEF740FE2749E06A0968C96AFB
:10655000884202D30120254908602048006808B914
:10656000012000E000200028D2D00CB1FEF764FB2F
:106570001F48056865B100BFFFF738FE10B1012064
:106580001A4908606D1E002DF6D1002018490860D8
:106590001648006838B10126300716490860BFF375
:1065A0004F8FBFF36F8FFEF75FFE304670BD000068
:1065B000280100202E2E5C4672656552544F535CB4
:1065C0007461736B732E63004572726F723A257338
:1065D0002C25640D0A000000000100205407002053
:1065E00008010020AC040020F0000020140100206D
:1065F0001001002004ED00E01CB50024FDF76AFF47
:106600000B48006858B10B481F2100234FF48072DB
:10661000CDE9001008A10A48FFF7A2FD04462CB9F5
:1066200040F2331207A10DA0FDF722F920461CBD50
:106630003401002038010020546D7220537663002D
:10664000C54D00082E2E5C4672656552544F535C52
:1066500074696D6572732E63000000004572726F7D
:10666000723A25732C25640D0A0000002DE9FE43C3
:1066700004460D4616461F46DDF828804FF00009F7
:106680002CB94FF4D37216A11BA0FDF7F1F81E48E8
:10669000006810B3009501960294062D15DAFFF7F5
:1066A0008FFD022808D1002342466946164800683B
:1066B000FFF774FB814610E000231A466946124832
:1066C0000068FFF76BFB814607E000233A46694606
:1066D0000D480068FFF758FC81464846BDE8FE8338
:1066E0002E2E5C4672656552544F535C74696D651D
:1066F00072732E63000000004572726F723A257348
:106700002C25640D0A00000034010020000303065C
:1067100001040602050003051F1C1F1E1F1E1F1F6C
:106720001E1F1E1F63757272656E74207061726128
:106730006D733A2025643A25642C686F74206F725B
:1067400020636F6C6420666C61673A25642C206856
:10675000756D696469747920666C61673A25642C8B
:1067600020616C61726D3A2025640D0A0000000002
:10677000256420202C25642020202C256420202026
:106780002C25642020202C25662020202C25662006
:10679000202C256620202C256620202C25662020F4
:1067A0002C256620202C256620202C252E33660DD6
:1067B0000A000000D467000800000020F00100007B
:1067C000500A000838680008F00100201832000064
:1067D000A03800081184A24A04400B0102030406F9
:1067E00007080917EF1CEEEE011A14FA02BC2A641E
:1067F00002FFFFFFFFEEEE0212FA0312FA0412FA92
:106800000512EA06120314B5050515FFFCFFFF0982
:106810001417256F12833AA3AA4329D269D60552C9
:10682000020406081AAA010128C30201B90D391190
:086830001A0314045D09D40CE5
:04000005080000ED02
:00000001FF
